:100000000C9453030C94E51F0C9412200C9484035D
:100010000C9484030C9484030C9484030C94840344
:100020000C9484030C9484030C9484030C94840334
:100030000C9484030C9484030C9484030C94840324
:100040000C943F200C9484030C943C220C948A2240
:100050000C9484030C9484030C9484030C94840304
:100060000C9467190C948403312E302E39005061A2
:1000700072616D65747261676500547970652064A2
:10008000652043686172676500436F7572616E74C5
:10009000204D6178696D756D0056657269662E2018
:1000A00064652044696F64650056657269662E2038
:1000B00056656E74205265712E0056657269662E03
:1000C000206465205465727265005265696E6974BA
:1000D00069616C6973657200536F72746965006160
:1000E000637469766500646573616374697665003D
:1000F000496E697469616C69736174696F6E0056E9
:100100006572696669636174696F6E0044657465E0
:10011000632E204175746F2E004E69766561753AC5
:10012000204E31004E69766561753A204E320045A9
:10013000525245555220455653450056454E544956
:100140004C2E2052455155495345004552522E20C0
:1001500056455249462044494F4445004552522E87
:1001600020444946464552454E54492E005041537D
:100170002044452054455252450052454C414920A7
:10018000424C4F51554500417272657465005645A9
:1001900020436F6E6E65637465005645204E6F6E2A
:1001A00020436F6E6E65637465006F6E00526573F9
:1001B000657474696E672E2E2E002000207020005A
:1001C0002D3E0073746174653A2000536574537654
:1001D000634C6576656C3A200020202000566572DD
:1001E00073696F6E20004F70656E20455653452031
:1001F000202020202020004F70656E5F455653451B
:100200003E2000556E6B6E6F776E20436F6D6D6193
:100210006E64202D2D2074797065203F206F722030
:1002200068656C7020666F7220636F6D6D616E64BF
:10023000206C69737400536176696E67205365742E
:1002400074696E677320746F20454550524F4D009E
:100250007361766500410043757272656E74204368
:1002600061706163697479206E6F773A2000496E1E
:1002700076616C69642043757272656E74204361A7
:1002800070616369747900293A20002D00456E740D
:10029000657220616D7073202800475245415445B6
:1002A00052205448414E2054484520524154454420
:1002B0002056414C5545204F462054484520455630
:1002C0005345004F4620594F5552204349524355FC
:1002D000495420425245414B4552204F520057410C
:1002E000524E494E47202D20444F204E4F5420530C
:1002F00045542043555252454E542048494748459D
:1003000052205448414E2038302500616D700073F2
:100310007475636B2072656C617920636865636BCB
:100320002000726C7963686B200067726F756E6471
:1003300020636865636B2000676E6463686B2000F0
:1003400064696F646520636865636B200064696F2E
:1003500063686B200076656E7420726571756972D2
:1003600065642000766E7472657120007365726931
:10037000616C20646562756767696E6720007364ED
:1003800062672000736574200073646267206F6E7B
:100390002F6F6666202D207475726E2073657269EA
:1003A000616C20646562756767696E67206F6E2F88
:1003B0006F666600726C7963686B206F6E2F6F6674
:1003C00066202D207475726E20737475636B2072B5
:1003D000656C617920636865636B206F6E2F6F6653
:1003E0006600676E6463686B206F6E2F6F666620B1
:1003F0002D207475726E2067726F756E642063684D
:1004000065636B206F6E2F6F66660064696F63684B
:100410006B206F6E2F6F6666202D20656E61626C9B
:10042000652F64697361626C652064696F6465201F
:10043000636865636B00766E74726571206F6E2FF2
:100440006F6666202D20656E61626C652F6469732E
:1004500061626C652076656E742072657175697273
:10046000656420737461746500616D7020202D20B7
:1004700053657420455653452043757272656E74FA
:100480002043617061636974790053657420436F20
:100490006D6D616E6473202D2055736167653A2020
:1004A00073657420616D70007365740073617665A7
:1004B000202D2057726974652073657474696E67A6
:1004C0007320746F20454550524F4D0073686F770D
:1004D000202D20446973706C617920736574746990
:1004E0006E677320616E642076616C75657300734E
:1004F000657420202D204368616E67652053657404
:1005000074696E67730068656C70202D2044697390
:10051000706C617920636F6D6D616E647300486506
:100520006C7020436F6D6D616E6473003F00686591
:100530006C7000537475636B2052656C6179204355
:100540006865636B3A200047726F756E642043687C
:1005500065636B3A200044696F6465204368656396
:100560006B3A200056656E7420526571756972652C
:10057000643A20004D61782043757272656E742074
:1005800043617061636974793A20004D696E20435C
:10059000757272656E742043617061636974793A33
:1005A000200043757272656E7420636170616369C7
:1005B00074792028416D7073293A20005365727652
:1005C000696365206C6576656C3A200053657474C8
:1005D000696E67730073686F77004F70656E5F4573
:1005E0005653453E200074797065203F206F72207D
:1005F00068656C7020666F7220636F6D6D616E64EC
:10060000206C69737400536F667477617265202D76
:10061000204F70656E204556534520004861726436
:1006200077617265202D2041746D656C2041544DB9
:10063000454741333238502D4155004F70656E208B
:10064000455653450000000000240027002A000002
:10065000000000250028002B0000000000230026D9
:100660000029000404040404040404020202020237
:100670000203030303030301020408102040800166
:1006800002040810200102040810200000000700E6
:10069000020100000304060000000000000000004A
:1006A000FD100318F62311241FBECFEFD8E0DEBFE4
:1006B000CDBF14BE88E10FB6F8948093600010920D
:1006C00060000FBE12E0A0E0B1E0E8EBFCE402C085
:1006D00005900D92A035B107D9F714E0A0E5B2E07E
:1006E00001C01D92AA3BB107E1F716E0C6EAD6E0C9
:1006F00004C02297FE010E941F26C03AD107C9F705
:100700000E944C240C945A260C940000FB01DC013E
:100710008D91059080190110D9F3990B0895FB0173
:10072000DC0105900D920020E1F70895FB01DC014A
:100730004150504030F08D910590801919F40020FF
:10074000B9F7881B990B0895FB01DC01415050401B
:1007500048F005900D920020C9F701C01D9241504C
:100760005040E0F70895AEE0B0E0E9EBF3E00C9420
:1007700031260D891E8986E08C831A8309838FEFC9
:100780009FE79E838D839E01275E3F4FCE0101969A
:100790006F89788DA9010E94D7032F813885020FB8
:1007A000131FF80110822E96E4E00C944D26ABE066
:1007B000B0E0EDEDF3E00C9423263C012B015A014F
:1007C000FC0117821682838181FD03C06FEF7FEFEA
:1007D000C6C19AE0892E1E010894211C311CF30128
:1007E0002381F20123FD859123FF81912F0188232D
:1007F00009F4B2C1853239F423FD859123FF81913B
:100800002F01853229F490E0B3010E94CA05E7CF99
:10081000982FFF24EE249924FFE1FF15D0F09B329E
:1008200069F09C3228F4903259F0933291F40EC062
:100830009D3249F0903369F441E024C052E0F52A3A
:1008400084E0F82A28C098E0F92A25C0E0E1FE2AD1
:1008500022C0F7FC29C0892F80538A3070F4F6FE3D
:1008600005C0989C902C1124980E15C0E89CE02C93
:100870001124E80EF0E2FF2A0EC09E3229F4F6FCA5
:100880006BC140E4F42A07C09C3619F450E8F52AFD
:1008900002C0983649F4F20123FD959123FF91910E
:1008A0002F01992309F0B8CF892F8554833018F090
:1008B0008052833038F444E050E0A40EB51E5FE36C
:1008C00059830FC0933631F0933779F0933509F09F
:1008D00056C020C0F5018081898342E050E0A40E1B
:1008E000B51E610101E010E012C0F501C080D180A9
:1008F000F6FC03C06FEF7FEF02C0692D70E042E0AD
:1009000050E0A40EB51EC6010E94BF058C015FE732
:10091000F52214C0F501C080D180F6FC03C06FEF52
:100920007FEF02C0692D70E042E050E0A40EB51EDA
:10093000C6010E94B4058C0150E8F52AF3FE07C0F9
:100940001AC080E290E0B3010E94CA05EA948E2D9D
:1009500090E008171907A8F30EC0F601F7FC85917F
:10096000F7FE81916F0190E0B3010E94CA05E1108A
:10097000EA94015010400115110579F7EAC0943648
:1009800011F0993669F5F7FE08C0F5012081318133
:100990004281538184E090E00AC0F5018081918119
:1009A0009C01442737FD4095542F82E090E0A80E2B
:1009B000B91E9FE6F92257FF09C050954095309522
:1009C00021953F4F4F4F5F4FE0E8FE2ACA01B90122
:1009D000A1012AE030E00E94F605D82ED21840C0CE
:1009E000953729F41F2D1F7E2AE030E01DC01F2DF2
:1009F000197F9F3661F0903720F4983509F0ACC02C
:100A00000FC0903739F0983709F0A6C004C028E02D
:100A100030E00AC0106114FD146020E130E004C031
:100A200014FD166020E132E017FF08C0F501608177
:100A300071818281938144E050E008C0F50180819A
:100A40009181BC0180E090E042E050E0A40EB51E30
:100A5000A1010E94F605D82ED2188FE7F82EF122B8
:100A6000F6FE0BC05EEFF522D91438F4F4FE07C091
:100A7000F2FC05C08FEEF82202C01D2D01C0192D19
:100A8000F4FE0DC0FE01ED0DF11D8081803319F4DF
:100A900099EEF92208C01F5FF2FE05C003C08F2D3A
:100AA000867809F01F5F0F2DF3FC14C0F0FE0FC015
:100AB0001E1510F09D2C0BC09D2C9E0C911A1E2D06
:100AC00006C080E290E0B3010E94CA051F5F1E15B8
:100AD000C0F304C01E1510F4E11A01C0EE2404FF97
:100AE0000FC080E390E0B3010E94CA0502FF1DC061
:100AF00001FD03C088E790E00EC088E590E00BC0E0
:100B0000802F867891F001FF02C08BE201C080E265
:100B1000F7FC8DE290E0B3010E94CA0506C080E3B5
:100B200090E0B3010E94CA059A94D914C0F3DA94F4
:100B3000F101ED0DF11D808190E0B3010E94CA0525
:100B4000DD20A9F706C080E290E0B3010E94CA054B
:100B5000EA94EE20C1F743CEF30166817781CB01A1
:100B60002B96E2E10C943F26FC0105906150704009
:100B70000110D8F7809590958E0F9F1F0895FC0166
:100B80006150704001900110D8F7809590958E0FBC
:100B90009F1F08950F931F93CF93DF938C01EB0159
:100BA0008B8181FF1BC082FF0DC02E813F818C8114
:100BB0009D812817390764F4E881F9810193F9834D
:100BC000E88306C0E885F985802F0995892B31F4E3
:100BD0008E819F8101969F838E8302C00FEF1FEF4E
:100BE000C801DF91CF911F910F910895FA01AA27B3
:100BF000283051F1203181F1E8946F936E7F6E5F60
:100C00007F4F8F4F9F4FAF4FB1E03ED0B4E03CD00D
:100C1000670F781F891F9A1FA11D680F791F8A1FF0
:100C2000911DA11D6A0F711D811D911DA11D20D057
:100C300009F468943F912AE0269F11243019305D11
:100C40003193DEF6CF010895462F4770405D419302
:100C5000B3E00FD0C9F7F6CF462F4F70405D4A334F
:100C600018F0495D31FD4052419302D0A9F7EACF17
:100C7000B4E0A6959795879577956795BA95C9F746
:100C800000976105710508959B01AC010A2E069439
:100C90005795479537952795BA95C9F7620F731FF2
:100CA000841F951FA01D0895FC01CB0106978E9708
:100CB00080F489E190E09C01629FC001639F900DE8
:100CC000729F900D112466E070E00E94D42561505F
:100CD00005C0CB01C4974D97F8F461566623E1F047
:100CE0002FB7F89483E6809380008BE18093810096
:100CF00089EF90E09093890080938800862F90E0A0
:100D000090938B0080938A002FBF81E090E09383C3
:100D1000828320E030E002C021E030E0C901089584
:100D2000CF93DF93FC016830F8F0878980FD03C022
:100D300020E130E002C020E230E0862F90E028176A
:100D4000390794F062A7C0E0D0E0442349F08281E3
:100D50009381019729F462A5CF0170E00E945406A7
:100D6000CE01DF91CF91089588E082A7C1E0D0E065
:100D7000ECCFFC018481882319F425E532E01BC007
:100D8000813019F42AE532E016C0823019F423E6E6
:100D900032E011C0833019F428E632E00CC0843010
:100DA00019F42DE632E007C0853019F020E030E07C
:100DB00002C022E732E0C9010895EF92FF920F933B
:100DC0001F938C0179010E94ED1DC801B7010E949B
:100DD0009F251F910F91FF90EF9008950F931F9300
:100DE0008C01462F60E00E94ED1D60918901709199
:100DF0008A01C8010E949F251F910F910895CF93EA
:100E0000DF93EC018C818F5F8C83823008F01C8231
:100E100081E093E061E070E00E94EE06EC81F0E09A
:100E2000EE0FFF1FEC53FE4F2081318181E093E0F4
:100E300060E070E041E050E00E94DD06DF91CF917C
:100E40000895CF93DF93EC018C818F5F8C83823088
:100E500008F01C8281E093E061E070E00E94EE0601
:100E600081E093E060E041E00E94ED1D8091D502B9
:100E70009C8183FD03C0992319F008C0992331F0A8
:100E800081E093E060E071E00E949F25EC81F0E05A
:100E9000EE0FFF1FEC53FE4F6081718181E093E004
:100EA0000E949F25DF91CF910895CF93DF93EC01AE
:100EB0008C818F5F8C83823008F01C8281E093E00C
:100EC00061E070E00E94EE0681E093E060E041E0C6
:100ED0000E94ED1D8091D5029C8182FD03C0992363
:100EE00019F008C0992331F081E093E060E071E0EF
:100EF0000E949F25EC81F0E0EE0FFF1FEC53FE4FA8
:100F00006081718181E093E00E949F25DF91CF9104
:100F10000895CF93DF93EC018C818F5F8C838230B7
:100F200008F01C8281E093E061E070E00E94EE0630
:100F300081E093E060E041E00E94ED1D8091D502E8
:100F40009C8181FD03C0992319F008C0992331F0D9
:100F500081E093E060E071E00E949F25EC81F0E089
:100F6000EE0FFF1FEC53FE4F6081718181E093E033
:100F70000E949F25DF91CF910895CF93DF93EC01DD
:100F80008C818F5F8C83833008F01C8281E093E03A
:100F900061E070E00E94EE0681E093E060E041E0F5
:100FA0000E94ED1D8091D50280FD02C021E001C0AC
:100FB00022E030E08C8190E001962817390731F467
:100FC00081E093E060E071E00E949F25EC81F0E019
:100FD000EE0FFF1FE955FE4F6081718181E093E0C4
:100FE0000E949F25DF91CF9108950F931F938C014D
:100FF00081E093E060E070E041E050E020E031E02B
:101000000E94DD06D8011496EC91F0E0EE0FFF1F70
:10101000EC53FE4F6081718181E093E00E949F2537
:10102000F80184818823C1F48091D502877F809361
:10103000D50287E293E062E070E04091D5020E9421
:10104000BD1764EF71E080E090E00E94952080E59C
:1010500092E01F910F9108958091D5028860E7CFAB
:101060000F931F938C0181E093E060E070E041E01A
:1010700050E020E031E00E94DD06D8011496EC91AA
:10108000F0E0EE0FFF1FEC53FE4F6081718181E0B5
:1010900093E00E949F25F80184818823C1F4809108
:1010A000D5028B7F8093D50287E293E062E070E007
:1010B0004091D5020E94BD1764EF71E080E090E09E
:1010C0000E94952080E592E01F910F9108958091F4
:1010D000D5028460E7CF0F931F938C0181E093E0EA
:1010E00060E070E041E050E020E031E00E94DD0689
:1010F000D8011496EC91F0E0EE0FFF1FEC53FE4F79
:101100006081718181E093E00E949F25F8018481D4
:101110008823C1F48091D5028D7F8093D50287E228
:1011200093E062E070E04091D5020E94BD1764EF49
:1011300071E080E090E00E94952080E592E01F91B0
:101140000F9108958091D5028260E7CF8091D502FA
:1011500080FD02C081E001C082E060E070E081308B
:1011600011F061E070E087E293E04091E8020E94B4
:10117000BD1787E293E062E070E04091D5020E94E3
:10118000BD170895CF92DF92EF92FF920F931F93B6
:10119000DF93CF93CDB7DEB769970FB6F894DEBF74
:1011A0000FBECDBF6C01262F7A0160E0422F0E9456
:1011B000ED1D00D000D000D0EDB7FEB731968E0106
:1011C0000F5F1F4FADB7BEB712961C930E931197CA
:1011D00082E091E093838283F582E4820E94B303EC
:1011E000198A8DB79EB706960FB6F8949EBF0FBEAC
:1011F0008DBFC601B8010E949F2569960FB6F8946D
:10120000DEBF0FBECDBFCF91DF911F910F91FF9039
:10121000EF90DF90CF900895EF92FF920F931F937E
:101220008C019B017A0160E070E0A9010E94C20874
:10123000C80161E070E0A7010E94C2081F910F91F0
:10124000FF90EF900895FC0114824091C4015091E9
:10125000C50181E093E068E071E00E940C09089507
:101260000F931F93CF93DF93EC011C828091D502E3
:1012700080FD04C08DEA91E041E003C084EB91E081
:1012800042E098878F831D821E8202C09F5F9E83EB
:10129000AF81B8859E81FD01E90FF11D8081882312
:1012A000A9F7292F21502E83A20FB11D8C918D8378
:1012B0003091E80290E0EF81F885E90FF11D80811F
:1012C000831711F49C8303C09F5F2917A0F7413057
:1012D00019F027E131E002C02AE131E000D000D06E
:1012E00000D0EDB7FEB731960EE712E0ADB7BEB74E
:1012F00012961C930E9311978DE191E09383828354
:10130000358324830E94B303EDB7FEB736960FB63C
:10131000F894FEBF0FBEEDBF81E093E060E070E0A7
:10132000A8010E94C20800D000D000D0ADB7BEB75F
:101330001196EDB7FEB7128301838CE291E013960C
:101340009C938E9312978C81EF81F885E80FF11DA5
:10135000808114968C93149715961C920E94B30367
:101360008DB79EB706960FB6F8949EBF0FBE8DBF81
:1013700081E093E061E070E0A8010E94C208DF9183
:10138000CF911F910F910895CF93DF93EC0181E0EE
:1013900093E060E070E041E050E020E031E00E9446
:1013A000DD068C81EF81F885E80FF11D608181E019
:1013B00093E070E04AE050E00E946D2581E093E008
:1013C00061E371E00E949F2564EF71E080E090E0AE
:1013D0000E9495208091D50280FD02C081E001C06D
:1013E00082E060E070E0813011F061E070E08C81BB
:1013F000EF81F885E80FF11D87E293E040810E94BC
:10140000BD178C81EF81F885E80FF11D8EEB92E01E
:10141000608140E00E94900680E592E0DF91CF91EC
:101420000895CF93DF93EC018C818F5F8C839E8135
:10143000981708F41C8281E093E061E070E00E945C
:10144000EE0681E093E060E041E00E94ED1D8C81BA
:10145000EF81F885E80FF11D9091E80280819817DF
:1014600031F481E093E060E071E00E949F258C817F
:10147000EF81F885E80FF11D608181E093E070E075
:101480004AE050E00E946D2581E093E061E371E065
:101490000E949F25DF91CF910895CF93DF93EC01B8
:1014A00081E093E00E94741E80FF52C031E00AC0C8
:1014B00089819A81AB81BC810097A105B10509F4AE
:1014C000188230E02881222361F0213009F045C0E4
:1014D00089819A81AB81BC810097A105B10509F48E
:1014E0003CC0332381F189819A81AB81BC81009713
:1014F000A105B10541F4222331F40E9487206983BC
:101500007A838B839C830E9487209B01AC01898115
:101510009A81AB81BC81281B390B4A0B5B0B8881FC
:10152000882339F42436310541055105B4F081E0B2
:1015300008C0813091F4245F3140404050406CF04D
:1015400082E088830AC019821A821B821C8205C02D
:101550008881823009F0B5CFABCFDF91CF9108956C
:101560000F931F938C018AE061E00E945521E1E80E
:10157000F6E0E491D801EC93EDE6F6E0E491119603
:10158000EC938E2F90E0880F991F815B994FFC019F
:10159000A591B4912FB7F894109280008C91F80126
:1015A0009081892B8C932FBF138212821F910F91F0
:1015B000089581E160E00E94552181E161E00E948F
:1015C000942108950F931F938C0188E060E00E949E
:1015D0009421F801808D8F7B808F0E947D1CF80103
:1015E00067AB70AF81AF92AF0E948720F80167A709
:1015F00070AB81AB92AB1F910F9108958091D60291
:1016000080688093D60286ED92E048970E94E20AB5
:101610008091BF0290E0880F991F815B994FFC0178
:10162000A591B4912FB7F894109280009C9180916D
:10163000BE02809598239C932FBF82E090E0909308
:10164000C1028093C00281E08093C20208950F938B
:101650001F938C0188E061E00E949421F801808D45
:101660008064808F0E947D1CF80163AB74AB85ABF6
:1016700096AB0E948720F80163A774A785A796A759
:101680001F910F910895DC015996EBE8F1E08AE093
:1016900001900D928150E1F70895CF92DF92EF9281
:1016A000FF920F931F938C017B016A01FC018685D9
:1016B0009785B9010E948F03F80126853785C801F7
:1016C000B701A6010E94DD061F910F91FF90EF90D8
:1016D000DF90CF900895EF92FF920F931F938C01AC
:1016E0007B01FC0186859785BA010E948F03F80172
:1016F00046855785C801B7010E94C2081F910F9106
:10170000FF90EF9008950F931F938C0181E093E079
:1017100060E070E041E050E020E031E00E94DD0652
:10172000D8011496EC91F0E0EE0FFF1FEC53FE4F42
:101730006081718181E093E00E949F2564EF71E0F8
:1017400080E090E00E949520F80184818823A1F434
:1017500081E093E061E070E04DEA51E00E946B0BA4
:101760002EE088E190E00FB6F894A8958093600091
:101770000FBE20936000FFCF80E090E01F910F919B
:101780000895EF92FF920F931F938C0131E0E32EA7
:1017900033E0F32EFC0142815381C70160E070E029
:1017A0000E946B0B8091D50290E023E0969587957F
:1017B0002A95E1F78170F801848300D000D000D031
:1017C000ADB7BEB711960EE712E0EDB7FEB71283C4
:1017D000018323E331E013963C932E931297E82F75
:1017E000F0E0EE0FFF1FEC53FE4F808191811596C4
:1017F0009C938E9314970E94B3038DB79EB7069661
:101800000FB6F8949EBF0FBE8DBFC70161E070E0B8
:10181000A8010E94C2081F910F91FF90EF900895B8
:10182000EF92FF920F931F938C0161E0E62E63E02D
:10183000F62EFC0142815381C70160E070E00E94F6
:101840006B0B8091D50290E096958795969587953C
:101850008170F801848300D000D000D0ADB7BEB74E
:1018600011960EE712E0EDB7FEB71283018323E372
:1018700031E013963C932E931297E82FF0E0EE0F91
:10188000FF1FEC53FE4F8081918115969C938E93A0
:1018900014970E94B3038DB79EB706960FB6F894BF
:1018A0009EBF0FBE8DBFC70161E070E0A8010E941E
:1018B000C2081F910F91FF90EF900895EF92FF9251
:1018C0000F931F938C01F1E0EF2EF3E0FF2EFC014C
:1018D00042815381C70160E070E00E946B0B8091F0
:1018E000D50290E0969587958170F801848300D0A9
:1018F00000D000D0ADB7BEB711960EE712E0EDB73D
:10190000FEB71283018323E331E013963C932E93B9
:101910001297E82FF0E0EE0FFF1FEC53FE4F80818F
:10192000918115969C938E9314970E94B3038DB763
:101930009EB706960FB6F8949EBF0FBE8DBFC70127
:1019400061E070E0A8010E94C2081F910F91FF9012
:10195000EF9008950F931F93CF93DF93EC014A818B
:101960005B8181E093E060E070E00E946B0B80910E
:10197000D50285FD02C01C8206C080FD02C081E048
:1019800001C082E08C8300D000D000D0ADB7BEB7DC
:1019900011960EE712E0EDB7FEB71283018383E3E1
:1019A00091E013969C938E931297EC81F0E0EE0FEA
:1019B000FF1FE955FE4F8081918115969C938E9370
:1019C00014970E94B3038DB79EB706960FB6F8948E
:1019D0009EBF0FBE8DBF81E093E061E070E0A80183
:1019E0000E94C208DF91CF911F910F910895FC01D1
:1019F00084818F5F8483873008F0148284818230F1
:101A0000D1F0833028F4882361F0813039F40EC09E
:101A10008430D9F08430A0F08530E1F048ED50E01A
:101A20001DC0409157025091580218C040915C026D
:101A300050915D0213C040916502509166020EC044
:101A400040916A0250916B0209C040916F0250911F
:101A5000700204C0409174025091750281E093E0DD
:101A600061E070E00E946B0B08950F931F93FC01DF
:101A7000148201E013E042815381C80160E070E00C
:101A80000E946B0B4091570250915802C80161E0CF
:101A900070E00E946B0B1F910F910895EF92FF92DF
:101AA0000F931F938C019B017A0160E070E0A90104
:101AB0000E946B0BC80161E070E0A7010E946B0BF4
:101AC0001F910F91FF90EF900895EF92FF920F9367
:101AD0001F93CF93DF93EC01898190E0880F991FCA
:101AE000815B994FFC01A591B4912FB7F8941092A6
:101AF00080008C919881892B8C932FBF1B821A8236
:101B000085E061E00E94942181E093E060EF70E065
:101B10004FEF50E00E944E0D8F8985FD57C081E048
:101B20000E943321298130E0220F331F215B394F7E
:101B3000F901A591B4914FB7F894109280003C91AF
:101B40002881209532233C934FBF22E030E03B8335
:101B50002A8318161906D4F588E061E00E949421C2
:101B600064EF71E080E090E00E94952083E00E94A5
:101B7000E8218C0184E00E94E8217C0188E060E09B
:101B80000E949421012B91F4EF2881F481E093E0ED
:101B90006CE071E044E251E00E944E0D64EF71E0B0
:101BA00080E090E00E94952002E011C081E093E087
:101BB0006CE071E049E151E00E944E0D64EF71E08C
:101BC00080E090E00E94952001E001C000E085E007
:101BD00060E00E949421898190E0880F991F815BC9
:101BE000994FFC01A591B4912FB7F8941092800001
:101BF0008C919881892B8C932FBF1B821A82802F06
:101C0000DF91CF911F910F91FF90EF9008958F92E8
:101C10009F92AF92BF92CF92DF92EF92FF920F937B
:101C20001F93CF93DF93EC010091E1028091D502E5
:101C300080FD03C0EE24E39402C062E0E62E8091B2
:101C4000E202081709F452C1053009F4EFC006306A
:101C500080F4023009F45BC0033020F4013009F055
:101C60003DC114C0033009F494C0043009F036C1FA
:101C7000CBC0073009F400C1073008F4EBC00830CE
:101C800009F40CC10F3F09F029C11AC18DE061E0D0
:101C90000E94942185E060E00E949421CE0162E0E0
:101CA0000E943E1E2DB73EB7285030400FB6F89424
:101CB0003EBF0FBE2DBFEDB7FEB731960EE712E067
:101CC000ADB7BEB712961C930E93119785E991E0BC
:101CD00093838283E48215828091E802868317824F
:101CE0000E94B3032DB73EB7285F3F4F0FB6F8945D
:101CF0003EBF0FBE2DBFCE0160E070E0A8010E9484
:101D0000C208CE0161E070E04AE951E03FC08DE0D9
:101D100061E00E94942185E061E00E949421CE015F
:101D200063E00E943E1E8DB79EB708970FB6F894E9
:101D30009EBF0FBE8DBFEDB7FEB731960EE712E026
:101D4000ADB7BEB712961C930E93119785E991E03B
:101D500093838283E48215828091E80286831782CE
:101D60000E94B3032DB73EB7285F3F4F0FB6F894DC
:101D70003EBF0FBE2DBFCE0160E070E0A8010E9403
:101D8000C208CE0161E070E04EE851E00E946B0BAA
:101D9000FFC08DE060E00E94942185E060E00E9439
:101DA0009421CE0164E00E943E1E8DB79EB7089735
:101DB0000FB6F8949EBF0FBE8DBFEDB7FEB731963C
:101DC0000EE712E0ADB7BEB712961C930E931197B3
:101DD00087E391E093838283E48215828091E80215
:101DE000868317820E94B3032DB73EB7285F3F4F0B
:101DF0000FB6F8943EBF0FBE2DBFCE0160E070E07D
:101E0000A8010E94C20875C08DE060E00E94942184
:101E100085E061E00E949421CE0161E00E943E1EB7
:101E2000CE016FE271E04BE351E011C08DE060E064
:101E30000E94942185E061E00E949421CE0161E03E
:101E40000E943E1ECE016FE271E04BE451E00E9421
:101E50004E0D9EC08DE060E00E94942185E061E01F
:101E60000E949421CE0161E00E943E1ECE016FE2ED
:101E700071E04CE551E0EBCF8DE060E00E949421F1
:101E800085E061E00E949421CE0161E00E943E1E47
:101E9000CE016FE271E04DE651E0D9CF8DE060E018
:101EA0000E94942185E061E00E949421CE0161E0CE
:101EB0000E943E1ECE016FE271E04AE751E0C7CFBB
:101EC0008DE060E00E94942185E061E00E94942111
:101ED000CE0160E070E047E851E058CF8DE060E06F
:101EE0000E94942185E061E00E949421033009F072
:101EF0004FC08090F9029090FA02A090FB02B0903F
:101F0000FC028091FD029091FE02A091FF02B0912F
:101F1000000388169906AA06BB06D1F1C501B401D3
:101F20000E944A1C6C01C501B4010E94441C7C0142
:101F3000C501B4010E943E1CADB7BEB71A970FB6DB
:101F4000F894BEBF0FBEADBFEDB7FEB731960EE73A
:101F500012E012961C930E93119729E431E033831B
:101F60002283D582C482F782E682918780870E948D
:101F7000B3032DB73EB7265F3F4F0FB6F8943EBF71
:101F80000FBE2DBFCE0161E070E0A8010E94C20823
:101F9000DF91CF911F910F91FF90EF90DF90CF9045
:101FA000BF90AF909F908F9008950F931F938C01D7
:101FB0008FEFF80183A3C8010E94E20AF801818132
:101FC00090E0880F991F815B994FFC01A591B49116
:101FD0002FB7F894109280009C91F8018081809531
:101FE00098239C932FBF82E090E09383828381E0CB
:101FF00093E00E94070E8FEFF80184A31F910F91C9
:1020000008950F931F93CF93DF93EC010E944D0A25
:102010008881813079F489819A81AB81BC81009774
:10202000A105B10509F07BC01882AD81BE81109772
:1020300029F475C0823009F072C009C0ED91FC919D
:1020400011970280F381E02DCD01099568C0898147
:102050009A81AB81BC810097A105B10509F45FC0ED
:1020600019821A821B821C82AD81BE81109709F4ED
:1020700046C0ED91FC9111970480F581E02DCD01D2
:102080000995DC019E838D830097D9F082E0A0350D
:10209000B80719F414960C911497ED91FC911197CF
:1020A0000190F081E02DCD010995ED81FE8182E066
:1020B000E035F807A1F501500483CF010E94F70C29
:1020C0002EC08FEF8093E2021092E1028091BF0256
:1020D00090E0880F991F815B994FFC01A591B49105
:1020E0002FB7F894109280008C919091BE02892BAA
:1020F0008C932FBF1092C1021092C00210C0809129
:10210000E1028250823058F08EEB92E00E94D50FAF
:1021100000E512E0C8010E94350D1E830D83DF919A
:10212000CF911F910F9108950F931F938C01FC0184
:10213000868597850E948F03F80166857785C8019B
:102140000E949F251F910F9108950F931F938C015B
:102150008DE061E00E94552185E061E00E945521FB
:102160008DE060E00E94942185E060E00E9494216F
:1021700081E0F8018587C80160E142E020E00E942B
:10218000A71EC80167E00E943E1EC80160E070E023
:1021900046EE51E00E946B0B64EF71E080E090E04E
:1021A0000E949520C80160E070E041E050E02DED14
:1021B00031E00E944D0BC80168E670E00E94941067
:1021C000C80169ED71E00E94941064EF71E080E055
:1021D00090E00E9495201F910F9108950F931F93F7
:1021E0008C0160E241E00E940C1D8EE792E0F80154
:1021F000978786871F910F9108958DE092E09093C5
:102200005102809350028EE690E0909353028093A7
:10221000520283E092E090935602809355028AE73F
:1022200090E0909358028093570289EF91E0909349
:102230005B0280935A0289E890E090935D0280935C
:102240005C028FEE91E0909364028093630289E9CF
:1022500090E0909366028093650285EE91E0909302
:1022600069028093680289EA90E090936B02809300
:102270006A028BED91E090936E0280936D028AEB7F
:1022800090E09093700280936F0281ED91E09093C3
:102290007302809372028AEC90E0909375028093AF
:1022A00074021092770210927802109279021092C2
:1022B0007A0210927B0210927D0210927C0281E0E1
:1022C00093E00E94EE1010922203109221038EE7F9
:1022D00092E0909324038093230380E490E0909312
:1022E00026038093250308950F931F938C01FC010F
:1022F00044895589828993890E94A403F8016289DF
:10230000738988E994E00E949F251F910F91089599
:102310006F927F929F92AF92BF92CF92DF92EF9295
:10232000FF920F931F93CF93DF93EC019BA02FEFAE
:10233000921639F465E070E080E090E00E9495200C
:1023400021C283E00E94E8218C0184E00E94E82100
:102350007C01888D86FF31C08F8983FD6FC00E940C
:1023600087202BA53CA54DA55EA5621B730B840B96
:10237000950B695E73408040904008F45FC0013067
:10238000110509F05BC0F1E0EF16F10409F056C049
:1023900087E08BA3CE010E94E20A8E898F3F11F065
:1023A0008F5F8E8B0E94872060567444824F9F4FB0
:1023B0006E877F87888B998BCEC127E0921609F5AF
:1023C0008A899B89AC89BD890397A105B10508F06D
:1023D000C0C10E9487202E853F8548895989621790
:1023E00073078407950708F4B4C18A899B89AC896F
:1023F000BD890196A11DB11D8A8B9B8BAC8BBD8BBA
:102400001DC08F8984FD1AC088E0981679F00E945B
:1024100087202FA538A949A95AA9621B730B840BE1
:10242000950B695E73408040904040F0012B11F0A5
:10243000EF2821F488E08BA318E08EC110E091E032
:102440008C818823D9F186E08BA389859A85AB8519
:10245000BC850397A105B10508F080C1F6E09F1681
:1024600051F08D858F3F11F08F5F8D8719861A8609
:102470001B861C8618C00E9487202D813E814F81BB
:102480005885621773078407950708F467C11C8293
:1024900089859A85AB85BC850196A11DB11D89876B
:1024A0009A87AB87BC870E94872060567444824F0E
:1024B0009F4F6D837E838F83988750C1992309F442
:1024C00081C0892D86508230B0F4898190E0880FD8
:1024D000991F815B994FFC01A591B4912FB7F89496
:1024E000109280008C919881892B8C932FBF1B8236
:1024F0001A821BA299241FEF612E13E0712EAA24C9
:10250000BB2400E010E081E00E943321A816B90648
:1025100014F45C0104C0861597050CF43C010F5FB0
:102520001F4F0436110579F7A5018F89682F81FDAA
:1025300017C18A819B81019709F012C189A19AA1D3
:102540006816790608F40CC115E015C08B8D9C8DBA
:102550002817390710F012E00EC08D8D9E8D2817B8
:10256000390740F462FF05C18F8D98A18217930748
:1025700008F0FFC013E0191529F18DA1181739F0E3
:102580000E9487206EA37FA388A799A71BC00E94E3
:102590008720CEA0DFA0E8A4F9A4113029F02AEF0B
:1025A00030E040E050E004C029E130E040E050E09D
:1025B0006C197D098E099F096217730784079507B7
:1025C00008F01BA31DA38BA1891509F4A5C08130B8
:1025D00079F0823049F1833049F46AA5CE0170E088
:1025E0000E945406CE010E94270B5DC08430C1F4C6
:1025F000CE010E94E20A898190E0880F991F815BD9
:10260000994FFC01A591B4912FB7F89410928000D6
:102610008C919881892B8C932FBF1B821A8243C087
:10262000863079F0853049F4CE010E94E20A6AA52D
:10263000CE0170E00E94540636C0873011F0883019
:10264000D9F4CE010E94E20A898190E0880F991F97
:10265000815B994FFC01A591B4912FB7F89410922A
:1026600080009C918881809598239C932FBF82E065
:1026700090E09B838A8317C0898190E0880F991F1F
:10268000815B994FFC01A591B4912FB7F8941092FA
:1026900080008C919881892B8C932FBF1B821A828A
:1026A000CE010E94E20A8F8987FF36C081E193E064
:1026B00063EC71E00E94741188E994E0692D70E088
:1026C0004AE050E00E946D2581E193E060EC71E00A
:1026D0000E9474116BA188E994E070E04AE050E038
:1026E0000E946D2581E193E06CEB71E00E94741112
:1026F00088E994E0B3014AE050E00E946D2581E151
:1027000093E06AEB71E00E94741188E994E0B501EE
:102710004AE050E00E9480259CA28BA1833091F575
:102720008BAD9CADADADBEADEF9688839983AA838A
:10273000BB83EF970E947D1C2BA93CA94DA95EA9E4
:10274000621B730B840B950B6BAF7CAF8DAF9EAF91
:1027500019C087E08BA317E090E072CE16E032CF6D
:102760009A01898D9A8D4817590708F4EFCE11E028
:1027700002CF8F8D98A18217930710F010E0FBCE47
:1027800014E0F9CEDF91CF911F910F91FF90EF9060
:10279000DF90CF90BF90AF909F907F906F90089503
:1027A0001F93CF93DF93EC01162F8F8987FF0EC005
:1027B00081E193E06BEC71E00E94741188E994E090
:1027C000612F70E04AE050E00E9480258F8912302E
:1027D00019F481608F8B03C08E7F8F8B11E060E0D6
:1027E00070E0113011F061E070E087E293E00E9448
:1027F000B617682F81508E3F20F01130E9F46FE05A
:1028000006C0683010F418E00BC0113029F4162F00
:10281000613130F010E104C0162F613208F010E28F
:10282000CE010E94430BCE01612F40E00E94900632
:10283000DF91CF911F91089560E1E7CFCF93DF93B0
:10284000EC016C81662321F48091D5028F7D07C055
:102850008EEB92E00E94D0138091D502806280932B
:10286000D50281E093E060E070E041E050E020E0DC
:1028700031E00E94DD06EC81F0E0EE0FFF1FE9552C
:10288000FE4F6081718181E093E00E949F2587E285
:1028900093E062E070E04091D5020E94BD1764EFC2
:1028A00071E080E090E00E94952080E592E0DF9169
:1028B000CF9108951F93CF93DF93EC0188E061E0FF
:1028C0000E94552183E060E00E94552184E060E091
:1028D0000E94552183E061E00E94942184E061E040
:1028E0000E949421CE010E94E20ACE010E94B00A09
:1028F00087E293E062E070E00E94B6178F3F11F428
:102900001F8A03C08F8B80FD02C011E001C012E05E
:10291000188E19861A861B861C861D861A8A1B8AA3
:102920001C8A1D8A1E8A1BA21CA2CE010E94650D54
:102930008111182FCE01612F0E94D0131C828DE0CF
:1029400060E00E949421DF91CF911F9108950F9331
:102950001F938C01FC0144895589828993890E94C7
:10296000A403F8016289738988E994E00E94A22592
:102970001F910F91089588E994E068E571E00E9445
:10298000A22508950F931F938C016BE376E00E94BC
:10299000A714C8016CE176E00E94A714C80166E0A4
:1029A00076E00E94A714C80168E670E00E94A714B0
:1029B000C8010E94BB141F910F9108950F931F939C
:1029C00010E00AE088E994E00E947D23982F90535C
:1029D0009A3020F4109F102D1124190F8D3091F78B
:1029E000812F1F910F9108950F931F93CF93DF9322
:1029F000EC0188E994E00E944C23892B09F45FC222
:102A000088E994E00E947D23182F88E994E0612FE3
:102A10000E9485241D30F9F0812F81568A3128F0DB
:102A20008F5C8A3010F0103241F488899989FE0158
:102A3000E80FF91F108301960BC0888999890097C8
:102A400009F42FC2183019F01F3709F02AC2019774
:102A5000998B888B26C2E889F989EC0FFD1F1082BB
:102A6000CE010E94BB14CE0165ED75E00E94860385
:102A7000892B09F086C0CE010E94C214CE016CECF5
:102A800075E00E94A714CE016CEB75E00E947411F2
:102A90008091D50280FD02C061E001C062E088E95A
:102AA00094E070E04AE050E00E948025CE0162EAA6
:102AB00075E00E9474116091E80288E994E070E08A
:102AC0004AE050E00E948025CE016BE875E00E944C
:102AD000741188E994E068E070E04AE050E00E94F8
:102AE0008025CE0164E775E00E94741188E994E0C6
:102AF00060E270E04AE050E00E948025CE0164E68A
:102B000075E00E9474118091D50282FF03C066EEC9
:102B100070E002C06FED70E0CE010E94A714CE01FC
:102B200066E575E00E9474118091D50281FF03C0B3
:102B300066EE70E002C06FED70E0CE010E94A71457
:102B4000CE0167E475E00E9474118091D50283FF85
:102B500003C066EE70E002C06FED70E0CE010E942F
:102B6000A714CE0163E375E00E9474118091D50231
:102B700084FF03C066EE70E002C06FED70E0CE012E
:102B80007BC1CE016EE275E00E948603892B41F085
:102B9000CE016CE275E00E948603892B09F086C1A4
:102BA000CE016EE175E00E94A714CE010E94BB1415
:102BB000CE0166E075E00E94A714CE016FEE74E0CE
:102BC0000E94A714CE016CEC74E00E94A714CE0101
:102BD0006CEA74E051C1CE016AE874E00E94A71467
:102BE000CE010E94BB14CE0169E674E00E94A714D6
:102BF000CE0166E374E00E94A714CE016BE074E09E
:102C00000E94A714CE0162EE73E00E94A714CE01C9
:102C100064EB73E00E94A714CE0169E873E02CC155
:102C2000CE0164E873E044E050E00E949603892BF3
:102C300009F010C18E010C5F1F4FC8016EE773E0F1
:102C400045E050E00E949603892BA9F4CE016CE682
:102C500073E00E947411CE0109966AEA71E00E9445
:102C60008603892B21F48091D502806859C0809118
:102C7000D5028F777CC0C80164E673E047E050E07E
:102C80000E949603892BA9F4CE0165E573E00E94AA
:102C90007411CE010B966AEA71E00E948603892BBB
:102CA00021F48091D5028B7F3BC08091D502846056
:102CB0005EC0C8016DE473E047E050E00E949603F7
:102CC000892BA9F4CE0160E473E00E947411CE0157
:102CD0000B966AEA71E00E948603892B21F48091A9
:102CE000D5028D7F1DC08091D502826040C0C80191
:102CF00068E373E047E050E00E949603892BD1F42B
:102D0000CE016AE273E00E947411CE010B966AEA6A
:102D100071E00E948603892B49F48091D502877F58
:102D20008093D502CE016FED70E0A6C08091D502F0
:102D300088601DC0C80162E273E047E050E00E9475
:102D40009603892BD1F4CE016FE073E00E947411D9
:102D5000C80107966AEA71E00E948603892B21F474
:102D60008091D5028F7EDCCF8091D50280618093E7
:102D7000D502CE0166EE70E07FC0C8016BE073E063
:102D80000E948603892B09F074C0CE016EED72E0BB
:102D90000E94A714CE0163EC72E00E94A714CE013A
:102DA0006AE972E00E94A714CE010E94BB14CE0112
:102DB0006DE872E00E94741188E994E068E070E0C8
:102DC0004AE050E00E946D25CE016BE872E00E945F
:102DD00074118091D50280FD03C060E170E002C0F3
:102DE00060E270E088E994E04AE050E00E946D25DE
:102DF000CE0167E872E00E947411CE010E94DE14D9
:102E0000182F88E994E0612F70E04AE050E00E94BA
:102E100080258EEB92E0612F41E00E949006892B85
:102E200029F0CE016EE672E00E94A714CE0167E59C
:102E300072E00E9474116091E80288E994E070E009
:102E40004AE050E00E946D25CE0165E572E00E94E7
:102E5000741114C0CE0160E572E00E948603892BD4
:102E600041F4CE0166E372E00E94A7140E94A60816
:102E700005C0CE0163E072E00E94A714CE010E945B
:102E8000BB14CE010E94BB14CE0167EF71E00E941B
:102E9000741188E994E00E94A623198A188A18827E
:102EA0000EC0888999890F9751F4D5CDCE0168EA73
:102EB00074E00E948603892B09F48DCEB1CEDF9198
:102EC000CF911F910F91089581E193E00E94F41436
:102ED0008EEB92E00E94881181E093E00E94070E41
:102EE00087E792E00E94011008950F931F938C01D1
:102EF0000E94C214C80166EE75E00E94A714C801C2
:102F00006AED75E00E94741188E994E00E94A6239E
:102F10001F910F91089581E093E00E94A5108EEB20
:102F200092E00E945A1481E193E00E94751708957F
:102F300088E10FB6F89480936000109260000FBE95
:102F400088E994E040E056E960E070E00E94C52224
:102F500080E06EEF7AE043E050E00E94C21F0E94E2
:102F60008B1787E792E00E94D90A0895F999FECF5E
:102F700072BD61BDF89A80B50895F999FECF1FBA68
:102F800072BD61BD40BD0FB6F894FA9AF99A0FBEB2
:102F9000089581E080936D0360934A0310926B0360
:102FA00010926C0308952091490330E0809148030A
:102FB000281B3109C90108954091480380914903B4
:102FC000481718F02FEF3FEF0AC0E42FF0E0E85D5C
:102FD000FC4F8081282F30E04F5F40934803C901A8
:102FE0000895E091480380914903E81718F0EFEF46
:102FF000FFEF06C0F0E0E85DFC4F8081E82FF0E0D5
:10300000CF0108950895109271031092700388EE15
:1030100093E0A0E0B0E08093720390937303A093D9
:103020007403B093750387E192E090936F038093EC
:103030006E030895CF92DF92EF92FF920F931F934A
:10304000CF93DF937C016B018A0180916D0388230C
:10305000A1F0C0E0D0E00DC0D701ED91FC91D60108
:10306000AC0FBD1F0190F081E02DC7016C91099557
:103070002196C017D10780F304C0CB01642F0E94B2
:103080004C19C801DF91CF911F910F91FF90EF90E4
:10309000DF90CF900895DF93CF930F92CDB7DEB737
:1030A000FC01698380916D038823C9F080916C03D2
:1030B000803238F081E090E09383828320E030E03A
:1030C00015C080916B03E82FF0E0E55BFC4F998120
:1030D00090838F5F80936B0380936C0305C0CE0158
:1030E000019661E00E944C1921E030E0C9010F9087
:1030F000CF91DF9108950F93062F80914A036BE4DF
:1031000073E040916C0321E00E94F71810926B036A
:1031100010926C0310926D030F91089561E00E946C
:103120007B180895413208F040E2862F68E273E090
:103130000E94AE181092480380934903089521E03D
:103140000E94921808951092480310924903109219
:103150006B0310926C030E94F81A0895382F4132C5
:1031600010F040E042C080917A038823E1F791E0BB
:1031700090937A0320937C038FEF8093E703109260
:10318000A20341504093A3034F5F90937B03809130
:103190007B03330F832B80937B0380917D038130EE
:1031A00041F410927D0380917B038093BB0085ECFA
:1031B00001C085EE8093BC0080917A038130E1F3F9
:1031C0008091A203841710F44091A20320E030E024
:1031D0000AC0FB01E20FF31FD901AE57BC4F8C911F
:1031E00080832F5F3F4F2417A0F3842F08950F9300
:1031F0001F93582F122F413210F081E04AC0809166
:103200007A038823E1F782E080937A0300937C03BA
:103210008FEF8093E7031092A2034093A303A2E8E9
:10322000B3E0FB0102C081918D938E2F861B841722
:10323000D0F310927B0380917B03550F852B8093F5
:103240007B0380917D03813041F410927D03809156
:103250007B038093BB0085EC01C085EE8093BC00AE
:10326000112321F080917A038230E1F38091E7030A
:103270008F3F11F480E00DC08091E703803211F49C
:1032800082E007C08091E703803311F084E001C041
:1032900083E01F910F910895482F613210F081E073
:1032A000089580917A03843011F082E0089560934C
:1032B000C503A4EAB3E0842F9C01F90102C0819107
:1032C0008D938E2F841B8617D0F380E008951F9274
:1032D0000F920FB60F9211242F933F934F935F934A
:1032E0006F937F938F939F93AF93BF93EF93FF93CE
:1032F0008091B90090E0887F90708036910509F444
:10330000F2C081369105CCF58832910509F47BC075
:1033100089329105B4F48031910509F46FC081318F
:1033200091053CF4009709F447C1089709F04FC193
:1033300065C08831910509F466C0809709F047C1DE
:1033400082C08034910509F4A4C08134910544F40D
:103350008033910509F482C0C89709F038C189C04B
:103360008035910509F489C08835910509F496C026
:103370008834910509F02BC1AEC08839910509F454
:1033800013C189399105ECF48837910509F4ABC074
:10339000893791054CF48836910509F4A4C080372B
:1033A000910509F014C19FC08838910509F4FCC04B
:1033B0008039910509F49DC08038910509F007C155
:1033C00098C0803B910509F4C6C0813B91054CF43F
:1033D000803A910509F49FC0883A910509F0F7C039
:1033E000BAC0803C910509F4E3C0883C910509F41A
:1033F000DFC0883B910509F0EAC0C2C080917B0321
:103400008093BB00CFC09091A2038091A303981733
:1034100068F49091A203E92FF0E0EE57FC4F808111
:103420008093BB009F5F9093A203BCC080917C03FC
:10343000882309F44BC085ED8093BC008091BC00CB
:1034400084FDFCCFC2C080E28093E70385ED8093CA
:10345000BC008091BC0084FDFCCFB7C080E38093AA
:10346000E70385ED8093BC008091BC0084FDFCCF18
:10347000ACC088E38093E7039BC08091A203909146
:10348000BB00E82FF0E0EE57FC4F90838F5F8093F6
:10349000A2039091A2038091A30382C08091A20312
:1034A0009091BB00E82FF0E0EE57FC4F90838F5FC8
:1034B0008093A20380917C03882341F085ED809363
:1034C000BC008091BC0084FDFCCF7FC081E0809374
:1034D0007D0384EA6EC085ED8093BC008091BC00C2
:1034E00084FDFCCF72C083E080937A031092E603E0
:1034F00059C08091E603803208F056C08091E603FF
:103500009091BB00E82FF0E0EA53FC4F90838F5F6F
:103510008093E60347C08091E603803230F4E09167
:10352000E603F0E0EA53FC4F108285ED8093BC0087
:103530008091BC0084FDFCCF10927A036091E60379
:10354000E0918003F091810386EC93E070E00995AF
:103550001092E6032DC084E080937A031092C40396
:103560001092C503E0917E03F0917F03099580914D
:10357000C503882329F481E08093C5031092A40336
:103580009091C403E92FF0E0EC55FC4F80818093CB
:10359000BB009F5F9093C4039091C4038091C503C7
:1035A000981710F485EC01C085E88093BC000FC02B
:1035B00085EC8093BC0009C01092E70385ED8093F1
:1035C000BC008091BC0084FDFCCF10927A03FF9177
:1035D000EF91BF91AF919F918F917F916F915F918B
:1035E0004F913F912F910F900FBE0F901F90189504
:1035F00010927A0381E080937C0310927D0382E134
:1036000061E00E94942183E161E00E949421E9EB52
:10361000F0E080818E7F808380818D7F808388E44D
:103620008093B80085E48093BC0008958F929F92A8
:10363000AF92BF92CF92DF92EF92FF920F931F93C0
:10364000CF93DF937B018C01EA012CE330E040E073
:1036500050E00E94E7256883C801B7012CE330E001
:1036600040E050E00E94E725122F032FF42EE52EB4
:10367000622F732F842F952F2CE330E040E050E031
:103680000E94E7256983612F702F8F2D9E2D2CE3DB
:1036900030E040E050E00E94E725122F032FF42E87
:1036A000E52E622F732F842F952F28E130E040E024
:1036B00050E00E94E7256A83612F702F8F2D9E2D89
:1036C00028E130E040E050E00E94E72579018A01DE
:1036D000C801B7016C5F7F4F8F4F9F4F27E030E0ED
:1036E00040E050E00E94E7256F5F6B83AA24BB2473
:1036F000650120E001C02F5F822E9924F401EE5471
:10370000F84FCF0183709070892B99F4CF0164E654
:1037100070E00E94D425892B39F4CF0160E971E073
:103720000E94D425892B29F48EE691E0A0E0B0E038
:1037300004C08DE691E0A0E0B0E0A80EB91ECA1E5C
:10374000DB1EC501A0E0B0E0E816F9060A071B077A
:1037500090F62E83F401EE54F84F83E0882E912CDE
:103760008E229F228114910499F4CF0164E670E0C7
:103770000E94D425892B39F4CF0160E971E00E94C1
:10378000D425892B29F48EE691E0A0E0B0E004C0B6
:103790008DE691E0A0E0B0E0A81AB90ACA0ADB0AF7
:1037A000980187010A191B092C093D09CF0164E61C
:1037B00070E00E94D4257C01CF0160E971E00E9495
:1037C000D425AC01E3E2F2E060E0613051F4811411
:1037D000910449F4E114F10441F44115510529F033
:1037E00002C0808103C08CE101C08DE190E0A0E0C7
:1037F000B0E0081719072A073B0740F0081B190B10
:103800002A0B3B0B6F5F31966C30F9F66F5F6D835F
:10381000802F8F5F8C83DF91CF911F910F91FF904D
:10382000EF90DF90CF90BF90AF909F908F900895D2
:10383000EF92FF920F931F937B018C018091FF0306
:1038400090910004A0910104B0910204E816F906D9
:103850000A071B0771F0C801B70144EF53E00E944B
:10386000161BE092FF03F0920004009301041093F2
:1038700002041F910F91FF90EF9008950E94181C71
:103880008091F40390E008950E94181C8091F50344
:1038900090E008950E94181C8091F60390E008952E
:1038A0006093EA037093EB038093EC039093ED0332
:1038B0002091C8013091C9014091CA015091CB01BA
:1038C000260F371F481F591F2093EE033093EF0335
:1038D0004093F0035093F10382E090E09093F30360
:1038E0008093F2030E9487206093FB037093FC0394
:1038F0008093FD039093FE030895EF92FF920F9340
:103900001F931CC02F5F3F4F4F4F5F4F2093EA0321
:103910003093EB034093EC035093ED0388EE93E078
:10392000A0E0B0E0E80EF91E0A1F1B1FE092FB03A7
:10393000F092FC030093FD031093FE030E94872086
:10394000E090FB03F090FC030091FD031091FE0357
:103950006E197F09800B910B2091EA033091EB03E4
:103960004091EC035091ED03685E734080409040BD
:1039700048F68091EE039091EF03A091F003B0918F
:10398000F103281739074A075B07C8F1E091E803FC
:10399000F091E903309799F1099561157105810559
:1039A000910519F00E94501C2AC08091C801909185
:1039B000C901A091CA01B091CB012091EA033091D5
:1039C000EB034091EC035091ED03820F931FA41F72
:1039D000B51F8093EE039093EF03A093F003B09391
:1039E000F10320E030E08091F2039091F303892B02
:1039F00011F021E030E03093F3032093F203609163
:103A0000EA037091EB038091EC039091ED031F9119
:103A10000F91FF90EF900895FC011382128283E3CF
:103A200092E091838083442311F481E001C082E01D
:103A300082876187148215860895682F8EE693E049
:103A40000E944B1808951F93162FFC016185606238
:103A50008EE693E070E00E94C91789E00E941D1D68
:103A6000812F0E941D1D8EE693E00E948E188823F0
:103A7000D1F71F9108951F93162FFC016185606295
:103A80008EE693E070E00E94C91783E10E941D1D3D
:103A9000812F0E941D1D8EE693E00E948E188823C0
:103AA000D1F71F910895DF92EF92FF920F931F932A
:103AB000CF93DF937C01062FD42EFC018585C62F82
:103AC000D0E08130A1F5648504FD6061C5FD6860CA
:103AD000C6FD646007FD6260DD2019F0162F106AD4
:103AE00002C0162F1062C701612F0E943B1D1F7D6F
:103AF000C701612F0E943B1DF7016485C0FD606115
:103B0000C1FD6860C2FD6460C3FD6260DD2019F024
:103B1000162F106A02C0162F1062C701612F0E9473
:103B20003B1D1F7DC701612F0E943B1D37C0D695ED
:103B3000C7959E012877442319F0922F966002C002
:103B4000922F9460F701858183FD02C010E001C0CF
:103B500010E8192BC701612F0E94231D1B7FC7018D
:103B6000612F0E94231D602F6F70660F660F660F16
:103B7000DD2011F0666001C06460F701858183FD7E
:103B800002C010E001C010E8162BC701612F0E948F
:103B9000231D1B7FC701612F0E94231DDF91CF9141
:103BA0001F910F91FF90EF90DF90089541E00E94E8
:103BB000531D81E090E0089540E00E94531D089558
:103BC000FC018285882341F06581862F846085838E
:103BD0006C60CF010E94DC1D0895DF93CF93CDB7B9
:103BE000DEB728970FB6F894DEBF0FBECDBF9C019D
:103BF000FC0182858823D9F0FE013196A7E3B2E06B
:103C000088E00D9001928150E1F7F90187818417D6
:103C100010F4482F4150E42FF0E0EE0FFF1FEC0F9F
:103C2000FD1F8181680F6068C9010E94DC1D289614
:103C30000FB6F894DEBF0FBECDBFCF91DF910895D0
:103C40000F931F93162F072FFC01618560628EE68C
:103C500093E070E00E94C91782E10E941D1D812F30
:103C60000E941D1D802F0E941D1D8EE693E00E9464
:103C70008E188823D1F71F910F910895FC0182853A
:103C8000882389F185858130F1F480EC91E0948777
:103C9000838760FF04C080E891E09487838761FF99
:103CA00005C0838594858F779487838762FF05C0DD
:103CB000838594859E7F9487838763857485CF01F0
:103CC0000E94201E08958581662311F0886001C03E
:103CD000877F8583858183FD02C060E001C060E845
:103CE000CF010E94231D0895CF93DF93EC018A85B5
:103CF0008823E9F0698560628EE693E070E00E94B7
:103D0000C91782E10E941D1D8EE693E00E948E1865
:103D1000698560628EE693E070E041E050E00E94C9
:103D20009F188EE693E00E94DC1780958F71DF91DB
:103D3000CF910895FC018285882341F0CF0161E095
:103D40000E94DC1D80ED97E00E94EE200895EF9226
:103D5000FF920F931F93DF93CF930F92CDB7DEB7F0
:103D60007C01042F122F62E370E080E090E00E945B
:103D700095208EE693E00E94A318F7018585618562
:103D8000813061F560628EE693E070E00E94C917B1
:103D900080E00E941D1D8FE10E941D1D8EE693E0B4
:103DA0000E948E18F701618560628EE693E070E0F4
:103DB0000E94C9178CE00E941D1D8FE10E941D1DED
:103DC0008EE693E00E948E18F701618560628EE6B0
:103DD00093E070E00E94C91781E034C060628EE613
:103DE00093E070E00E94C91780E00E941D1D8FEFD4
:103DF0000E941D1D80E00E941D1D80E00E941D1D6F
:103E000080E00E941D1D80E00E941D1D80E00E9438
:103E10001D1D80E00E941D1D80E00E941D1D80E090
:103E20000E941D1D80E00E941D1D8EE693E00E94F1
:103E30008E18F701618560628EE693E070E00E9463
:103E4000C91780E00E941D1D80E00E941D1D8EE6A6
:103E500093E00E948E18023020F0F7018481886080
:103E60008483F70107831086112329F0013019F4A8
:103E7000848184608483F7018285823091F4818516
:103E8000BE016F5F7F4F40E021E000E00E94F71825
:103E9000882321F481E0F701828703C0F7011286AD
:103EA00069C0F70185858130B9F41486138600E076
:103EB000C70168E30E943B1DC70168E10E943B1DEA
:103EC0000F5F0330A9F7C70168E20E943B1DC701DD
:103ED00068E00E943B1D20C0C7016CE90E94231DC1
:103EE000C70168E90E94231DC7016CE90E94231DD8
:103EF000C70168E90E94231DC7016CE90E94231DC8
:103F0000C70168E90E94231DC70164E90E94231DBF
:103F1000C70160E90E94231D65E070E080E090E049
:103F20000E949520F70164816062C7010E94DC1D38
:103F300065E070E080E090E00E949520F7016481E8
:103F40006062C7010E94DC1D65E070E080E090E0E7
:103F50000E9495208CE0F7018583C7010E94E01D37
:103F6000C7010E949A1E82E0F7018683C70166E0BE
:103F70000E94DC1D0F90CF91DF911F910F91FF9058
:103F8000EF900895823000F5E82FF0E0EE0FFF1F6C
:103F9000ED5FFB4F71836083882319F08130A1F4BA
:103FA00008C0809169008C7F842B80936900E89A17
:103FB000089580916900440F551F440F551F837F5A
:103FC000842B80936900E99A08951F920F920FB68F
:103FD0000F9211242F933F934F935F936F937F938F
:103FE0008F939F93AF93BF93EF93FF9380910304BD
:103FF00090910404892B29F0E0910304F0910404CA
:104000000995FF91EF91BF91AF919F918F917F9112
:104010006F915F914F913F912F910F900FBE0F9035
:104020001F9018951F920F920FB60F9211242F9385
:104030003F934F935F936F937F938F939F93AF9330
:10404000BF93EF93FF938091050490910604892B11
:1040500029F0E0910504F09106040995FF91EF9194
:10406000BF91AF919F918F917F916F915F914F9190
:104070003F912F910F900FBE0F901F9018951F9298
:104080000F920FB60F9211242F933F938F939F930C
:10409000AF93BF9380910B0490910C04A0910D04F9
:1040A000B0910E0430910F040196A11DB11D232F74
:1040B0002D5F2D3720F02D570196A11DB11D2093A6
:1040C0000F0480930B0490930C04A0930D04B09301
:1040D0000E048091070490910804A0910904B09106
:1040E0000A040196A11DB11D809307049093080452
:1040F000A0930904B0930A04BF91AF919F918F914F
:104100003F912F910F900FBE0F901F9018958FB772
:10411000F89420910B0430910C0440910D045091BF
:104120000E048FBFB901CA0108959B01AC017FB78E
:10413000F8948091070490910804A0910904B0912B
:104140000A0466B5A89B05C06F3F19F00196A11D32
:10415000B11D7FBFBA2FA92F982F8827860F911DD9
:10416000A11DB11D62E0880F991FAA1FBB1F6A9590
:10417000D1F7BC012DC0FFB7F8948091070490914E
:104180000804A0910904B0910A04E6B5A89B05C0F3
:10419000EF3F19F00196A11DB11DFFBFBA2FA92F46
:1041A000982F88278E0F911DA11DB11DE2E0880F69
:1041B000991FAA1FBB1FEA95D1F7861B970B885E34
:1041C0009340C8F2215030404040504068517C4FED
:1041D000211531054105510571F60895019739F012
:1041E000880F991F880F991F02970197F1F708957B
:1041F000789484B5826084BD84B5816084BD85B5C2
:10420000826085BD85B5816085BDEEE6F0E0808188
:1042100081608083E1E8F0E01082808182608083A9
:10422000808181608083E0E8F0E08081816080832C
:10423000E1EBF0E0808184608083E0EBF0E080815E
:1042400081608083EAE7F0E0808184608083808100
:1042500082608083808181608083808180688083A8
:104260001092C1000895982F8E3008F09E509770DC
:104270008091CC018295880F880F807C892B809358
:104280007C0080917A00806480937A0080917A002B
:1042900086FDFCCF2091780040917900942F80E03A
:1042A00030E0282B392BC9010895CF93DF93482F95
:1042B00050E0CA018958994FFC0134914D59594F2A
:1042C000FA018491882369F190E0880F991FFC011D
:1042D000EB5BF94FA591B491FC01E15BF94FC591FE
:1042E000D491662351F42FB7F8948C91932F909525
:1042F00089238C93888189230BC0623061F42FB7A6
:10430000F8948C91932F909589238C938881832B9B
:1043100088832FBF06C09FB7F8948C91832B8C9312
:104320009FBFDF91CF910895482F50E0CA01855774
:10433000994FFC012491CA018958994FFC0194912D
:104340004D59594FFA013491332309F440C02223C7
:1043500051F1233071F0243028F42130A1F02230C3
:1043600011F514C02630B1F02730C1F02430D9F453
:1043700004C0809180008F7703C0809180008F7D82
:104380008093800010C084B58F7702C084B58F7D84
:1043900084BD09C08091B0008F7703C08091B000C8
:1043A0008F7D8093B000E32FF0E0EE0FFF1FE15B05
:1043B000F94FA591B4912FB7F894662321F48C910D
:1043C0009095892302C08C91892B8C932FBF0895DF
:1043D000682F70E0CB018557994FFC012491CB01E8
:1043E0008958994FFC0144916D59794FFB01949183
:1043F000992319F420E030E03CC0222351F123300E
:1044000071F0243028F42130A1F0223011F514C0CD
:104410002630B1F02730C1F02430D9F404C08091A7
:1044200080008F7703C0809180008F7D8093800013
:1044300010C084B58F7702C084B58F7D84BD09C05C
:104440008091B0008F7703C08091B0008F7D809302
:10445000B000892F90E0880F991F875A994FFC016F
:10446000A591B4918C9120E030E0842311F021E0FB
:1044700030E0C901089508951F920F920FB60F9270
:1044800011242F933F934F938F939F93EF93FF9319
:104490008091C00082FD1DC04091C6002091500453
:1044A000309151042F5F3F4F2F7330708091520431
:1044B000909153042817390771F0E0915004F0915E
:1044C0005104E05FFB4F408330935104209350042C
:1044D00002C08091C600FF91EF919F918F914F9103
:1044E0003F912F910F900FBE0F901F901895E09164
:1044F000A404F091A504E05CFF4F8191919120818B
:104500003181821B930B8F739070892B11F00E9465
:104510003B2208951F920F920FB60F9211242F93F2
:104520003F938F939F93EF93FF9320919404309147
:10453000950480919604909197042817390731F4D7
:104540008091C1008F7D8093C10014C0E0919604DA
:10455000F0919704EC5AFB4F208180919604909142
:10456000970401968F7390709093970480939604AC
:104570002093C600FF91EF919F918F913F912F91D2
:104580000F900FBE0F901F901895AF92BF92DF92C1
:10459000EF92FF920F931F93CF93DF93EC017A0179
:1045A0008B01DD24403081EE580780E0680780E011
:1045B000780711F0DD24D39491E0A92EB12CEC8979
:1045C000FD89DD2069F0C50108A002C0880F991F90
:1045D0000A94E2F7808360E079E08DE390E005C023
:1045E000108260E874E88EE190E0A80197010E94D3
:1045F000E72521503040404050405695479537952B
:10460000279580E12030380720F0DD2011F0DD24EF
:10461000D6CFE889F9893083EA89FB89208319A2FA
:10462000EE89FF89408121E030E0C9010C8C02C095
:10463000880F991F0A94E2F7482B4083EE89FF897F
:104640004081C9010D8C02C0880F991F0A94E2F7BE
:10465000482B4083EE89FF894081C9010E8C02C03E
:10466000880F991F0A94E2F7482B4083EE89FF894F
:1046700080810F8C02C0220F331F0A94E2F720952D
:1046800028232083DF91CF911F910F91FF90EF900E
:10469000DF90BF90AF900895DC011C96ED91FC91E6
:1046A0001D97E05CFF4F2191319180819181281B02
:1046B000390B2F733070C9010895DC011C96ED9100
:1046C000FC911D97E05CFF4F20813181E054F04068
:1046D000DF01AE5BBF4F8D919C9111972817390771
:1046E00019F42FEF3FEF07C08D919C91E80FF91F50
:1046F0008081282F30E0C9010895DC011C96ED91DE
:10470000FC911D97E05CFF4F20813181E054F04027
:10471000DF01AE5BBF4F8D919C9111972817390730
:1047200019F42FEF3FEF10C08D919C911197E80F76
:10473000F91F20818D919C91119701968F73907034
:1047400011969C938E9330E0C9010895DC019196F7
:104750008C919197882339F05496ED91FC9155975F
:10476000808186FFF9CF91961C920895CF93DF93B5
:10477000EC01EE85FF85E05CFF4F20813181E05444
:10478000F0402F5F3F4F2F733070DF01AE5BBF4FA4
:104790008D919C91119728173907D1F3E05CFF4F59
:1047A00080819181E054F040E80FF91F6083EE852D
:1047B000FF85E05CFF4F31832083EE89FF892081F4
:1047C00081E090E00F8C02C0880F991F0A94E2F7F5
:1047D000282B208381E089A3EC89FD898081806476
:1047E000808381E090E0DF91CF91089510929B0447
:1047F00010929A0488EE93E0A0E0B0E080939C04CD
:1048000090939D04A0939E04B0939F0483E492E050
:10481000909399048093980480E194E09093A50488
:104820008093A40484E594E09093A7048093A60465
:1048300085EC90E09093A9048093A80484EC90E028
:104840009093AB048093AA0480EC90E09093AD0425
:104850008093AC0481EC90E09093AF048093AE041D
:1048600082EC90E09093B1048093B00486EC90E0E9
:104870009093B3048093B20484E08093B40483E003
:104880008093B50487E08093B60485E08093B704F5
:1048900081E08093B8040895CF93DF930E94F820BD
:1048A0000E949817C7E7D2E20E9464172097E1F3AD
:1048B0000E947722F9CFCF92DF92EF92FF920F936F
:1048C0001F93CF93DF937C016B018A01C0E0D0E09E
:1048D0000FC0D6016D916D01D701ED91FC91019052
:1048E000F081E02DC7010995C80FD91F0150104074
:1048F0000115110571F7CE01DF91CF911F910F9135
:10490000FF90EF90DF90CF900895DC01ED91FC9146
:104910000190F081E02D09950895EF92FF920F9399
:104920001F938C01DC01ED91FC910190F081E02D51
:104930006DE009957C01D801ED91FC910190F08129
:10494000E02DC8016AE009959C012E0D3F1DC901AB
:104950001F910F91FF90EF900895CF93DF93EC019B
:104960006115710519F420E030E00FC0DB010D90F6
:104970000020E9F71197A61BB70BE881F9810280A7
:10498000F381E02DAD0109959C01C901DF91CF9123
:1049900008954F925F927F928F929F92AF92BF92B3
:1049A000CF92DF92EF92FF920F931F93DF93CF93FB
:1049B000CDB7DEB7A1970FB6F894DEBF0FBECDBF5F
:1049C0002C01742ECB01223008F42AE019A231E226
:1049D000C32ED12CCC0EDD1E822E9924AA24BB24FA
:1049E000672D752FA50194010E94E72579018A01A1
:1049F000C801B701A50194010E94B525472D461BAA
:104A00000894C108D1084A3014F4405D01C0495CE3
:104A1000F6014083E114F1040105110521F07E2C1B
:104A20005F2DC801DDCFC201B6010E94AD24A19661
:104A30000FB6F894DEBF0FBECDBFCF91DF911F91AF
:104A40000F91FF90EF90DF90CF90BF90AF909F902D
:104A50008F907F905F904F900895CF92DF92EF926A
:104A6000FF920F931F93CF93DF93EC016A017B01B9
:104A70002115310541F4E881F9810190F081E02DA3
:104A8000642F09951FC02A303105D1F477FF17C074
:104A9000E881F9810190F081E02D6DE209958C01AA
:104AA00044275527BA014C195D096E097F09CE01CB
:104AB0002AE00E94C9249801280F391F04C02AE067
:104AC0000E94C9249C01C901DF91CF911F910F91D0
:104AD000FF90EF90DF90CF900895EF92FF920F93A9
:104AE0001F937B019A010027F7FC0095102FB80156
:104AF000A7010E942D251F910F91FF90EF9008951F
:104B0000CF92DF92EF92FF920F931F936C017B0184
:104B10009A010027F7FC0095102FB801A7010E9409
:104B20002D258C01C6010E948D24080F191FC80174
:104B30001F910F91FF90EF90DF90CF9008950E940A
:104B4000AD240895EF92FF920F931F937C010E9472
:104B5000AD248C01C7010E948D24080F191FC801C4
:104B60001F910F91FF90EF900895629FD001739F66
:104B7000F001829FE00DF11D649FE00DF11D929FF9
:104B8000F00D839FF00D749FF00D659FF00D992738
:104B9000729FB00DE11DF91F639FB00DE11DF91F5C
:104BA000BD01CF011124089597FB092E07260AD0D5
:104BB00077FD04D02ED006D000201AF470956195B0
:104BC0007F4F0895F6F7909581959F4F0895A1E244
:104BD0001A2EAA1BBB1BFD010DC0AA1FBB1FEE1F77
:104BE000FF1FA217B307E407F50720F0A21BB30BC2
:104BF000E40BF50B661F771F881F991F1A9469F73E
:104C000060957095809590959B01AC01BD01CF0199
:104C10000895AA1BBB1B51E107C0AA1FBB1FA61703
:104C2000B70710F0A61BB70B881F991F5A95A9F755
:104C300080959095BC01CD010895EE0FFF1F059062
:104C4000F491E02D09942F923F924F925F926F92D0
:104C50007F928F929F92AF92BF92CF92DF92EF920C
:104C6000FF920F931F93CF93DF93CDB7DEB7CA1B8D
:104C7000DB0B0FB6F894DEBF0FBECDBF09942A88B8
:104C8000398848885F846E847D848C849B84AA8460
:104C9000B984C884DF80EE80FD800C811B81AA81ED
:104CA000B981CE0FD11D0FB6F894DEBF0FBECDBFB8
:084CB000ED010895F894FFCF17
:104CB8002B00252D313673005265696E6974696160
:104CC8006C697365723F004C32004C3100257320CB
:104CD8004D61782043757272656E74002B256441AE
:104CE8000041002B2573004368617267696E672075
:104CF800204C25643A25644100253032643A253039
:104D080032643A2530326400002020202020202000
:104D1800202020202020202020004175746F004E84
:104D280069766561752031004E6976656175203256
:104D3800004F7569004E6F6E0059016B030C03B28A
:104D48000200000401507265742020202020204EAB
:104D580025643A256441006A016F017801060A0C4E
:104D68000E0F10000A1014191E23282D32373C414B
:104D7800464B5000810185012C0100000100000014
:104D8800002309FF06830B00000000C10B2107F573
:104D98000700000000100C55073008000000005EF6
:104DA8000C89076B08000000003009110AC40900CB
:104DB800000000AA0CBD071E1400000000350DF706
:104DC8000CB906000000004B181A18D317DC17F1AD
:104DD8001702181F1C1F1E1F1E1F1F1E1F1E1F002D
:104DE800000000D61D5B24000040001400540000A1
:104DF800000000B6235B244C237D235D23A62300FB
:00000001FF
